:100000000C9438010C9455010C9455010C94550135
:100010000C9455010C9455010C9455010C94550108
:100020000C9455010C9455010C9455010C945501F8
:100030000C9425130C9455010C9455010C94550106
:100040000C9455010C94FC050C94481B0C94341230
:100050000C94C4120C9455010C9455010C94550148
:100060000C9455010C9455010C9455010C945501B8
:100070004570692D4F5344205665722E302E392E0F
:10008000372E302E310000416B7475656C6C6573D2
:100090002053657474696E67000053657474696EEB
:1000A0006720200000486F6568656E73656E736F2A
:1000B000722000004853206D697420536368616C9E
:1000C00074657220000048656164696E6720486F3E
:1000D0006C642000004B6F6D706173732000004BE7
:1000E0006F6D70617373206669782000004750530C
:1000F00020416B74697620000041636873656E6B04
:100100006F7070656C756E67200000447265687270
:1001100061746520626567722E2000004665686C18
:1001200065722046433C2D3E4F5344200000556EDF
:100130007465727370616E6E756E672000004B653A
:10014000696E652053657474696E672D416E7A65BA
:10015000696765000050432F425420616B746976D3
:10016000000055656265726E65686D65204C65744A
:100170007A7465732053657474696E6700004B650B
:10018000696E65204465766976652D416E7A65698C
:100190006765000050432F425420616B74697600FC
:1001A0000055656265726E65686D65204C65747A90
:1001B0007465732044657669636500004F4E0000E6
:1001C0002D2D2D000044657669636520756E6420D1
:1001D00056657273696F6E736162667261676500FE
:1001E0000044657669636520202020203D200000C2
:1001F00046572D56657273696F6E203D200000468C
:100200004300004E43000046432D6F6C6420465768
:1002100000004550492D4D656E750050616C0050D1
:10022000432F4254004B656E6E756E670052432D2E
:1002300042657472696562004550492D5374726F4E
:100240006D0045786974004F4E002D2D0076767D47
:1002500076767A76767E76767776767B767678762A
:10026000767C76767976767D76767A76767E760088
:1002700011241FBECFEFD4E0DEBFCDBF11E0A0E060
:10028000B1E0E8E1F9E302C005900D92A239B107AF
:10029000D9F713E0A2E9B1E001C01D92A33FB10775
:1002A000E1F70E9465010C948A1C0C94000086E919
:1002B00081BB8FE084BBAC9AAD9A8EE28ABB80EBA7
:1002C00087BBC69AD99ADD9A08951092DA011092E6
:1002D000D6011092DB01E199FECF80E090E09FBB58
:1002E0008EBBE09A8DB380939901E199FECF81E0B6
:1002F00090E09FBB8EBBE09A8DB380930001E199A3
:10030000FECF82E090E09FBB8EBBE09A8DB38093DE
:100310009A01E199FECF87E190E09FBB8EBBE09A06
:100320008DB38093A701E199FECF88E190E09FBB58
:100330008EBBE09A8DB38093C001E199FECF8AE134
:1003400090E09FBB8EBBE09A8DB380930901E19949
:10035000FECF89E190E09FBB8EBBE09A8DB3809386
:10036000BC01E199FECF8BE190E09FBB8EBBE09A90
:100370008DB380939B0120910001213079F49EE0A0
:100380009093030187E08093040186E88093050140
:1003900020930601909307018CE00EC09CE090939F
:1003A000030185E0809304018AE4809305011092A3
:1003B0000601909307018AE0809308010E94421889
:1003C0000E9457010E94F50580919901813019F42E
:1003D0000E940F1102C00E94FF107894A89A0E94F8
:1003E0001B050E945C060E944F0A80919B01882396
:1003F00011F00E948F0A8091C501882311F00E949C
:1004000035140E948F0A80919B01813011F40E9463
:10041000981B0E94E0118091B801813021F4109264
:10042000B8010E94DA188091DF01813021F4109226
:10043000DF010E94250E809194018130C9F4109251
:1004400094018091DA01882369F48091BC018430A1
:1004500049F480919901882329F480E364E641E01E
:100460000E948E110E9418130E941D130E94851570
:1004700080919B01813031F48091E001813011F451
:100480000E94A31B809197018130E1F48091DA01F1
:100490008823C1F4AA9A0E94660F0E94AF090E94A5
:1004A000C4088091C301882321F00E9491130E9407
:1004B0000D0B8091C401882311F00E948A180E94BC
:1004C000E40AAA9880919201813009F03FC080919E
:1004D000DA018823D9F5109292018091BC01823013
:1004E00029F483E66FE64AE00E948E118091BC01F8
:1004F000813029F482E664E64AE00E948E11809100
:10050000A701882321F080910201833014F00E941A
:10051000BE0A8091A4019091A50101969093A50136
:100520008093A4010197CB9769F48091A2019091E7
:10053000A30101969093A3018093A2011092A501BB
:100540001092A4010E949D0C0E94E70D80919301DE
:10055000813009F060CF8091DA01882309F05BCF08
:100560001092930180919B01813039F48091E001D8
:10057000882319F481E00E94A31B0E94580A8091ED
:10058000C501882309F447CF0E9491140E941114D9
:100590000E94FC140E9462140E943D140E94F313F6
:1005A0003ACF782FD99827E030E041E050E0DB984F
:1005B0000000000000000000CA01022E02C0880FE7
:1005C000991F0A94E2F7872311F0DA9A01C0DA98AA
:1005D0000000000000000000DB9A000000000000A6
:1005E0000000215030408FEF2F3F380701F727E000
:1005F00030E041E050E0DB98000000000000000027
:10060000CA01022E02C0880F991F0A94E2F78623BE
:1006100011F0DA9A01C0DA98000000000000000032
:10062000DB9A0000000000000000215030408FEFF6
:100630002F3F380701F7DB98DA98D99A089584E0BC
:1006400064E00E94D10280E06CE40E94D10210922A
:100650009401809194018823E1F38CE66AE00E9482
:10066000D10285E060E00E94D10208950F931F93AC
:10067000809192018823E1F3109292018091BC0154
:10068000823051F40E941F111092920180919201C8
:100690008823E1F3109292011092C2010E94660F2A
:1006A00082E661E74FEF0E948E1110E000E01DC06E
:1006B00080919701813071F480917B02813519F42A
:1006C0000E94660F02C08091970182E661E74FEFBA
:1006D0000E948E1180919201813039F410E0023035
:1006E00009F411E0109292010F5F8091C2018823FA
:1006F00011F41123E9F28091BC01823011F40E94BF
:100700006611112309F0D9C08091E4038093090197
:100710008091CD038093C0012091C001E199FECF6B
:1007200088E190E09FBB8EBB2DBB0FB6F894E29A98
:10073000E19A0FBE20910901E199FECF8AE190E094
:100740009FBB8EBB2DBB0FB6F894E29AE19A0FBE09
:1007500082E061E047E850E00E94A10E82E062E0A2
:100760004AE950E00E94A10E82E064E045EA50E0D0
:100770000E94A10E82E065E044EB50E00E94A10ED1
:1007800082E066E046EC50E00E94A10E82E067E065
:1007900045ED50E00E94A10E82E068E04FED50E090
:1007A0000E94A10E82E069E04DEE50E00E94A10E91
:1007B00082E06AE049EF50E00E94A10E82E06BE027
:1007C0004EE251E00E94A10E4091BE015091BF0146
:1007D00084E162E00E94FA0D8091C00180FF05C0B3
:1007E00084E164E04CEB51E004C084E164E040EC5F
:1007F00051E00E94A10E8091C00181FF05C084E1FB
:1008000065E04CEB51E004C084E165E040EC51E070
:100810000E94A10E8091C00182FF05C084E166E0C4
:100820004CEB51E004C084E166E040EC51E00E94F2
:10083000A10E8091C00183FF05C084E167E04CEB0D
:1008400051E004C084E167E040EC51E00E94A10E59
:100850008091C00184FF05C084E168E04CEB51E069
:1008600004C084E168E040EC51E00E94A10E809158
:10087000C00185FF05C084E169E04CEB51E004C094
:1008800084E169E040EC51E00E94A10E8091C0013A
:1008900086FF05C084E16AE04CEB51E004C084E1CE
:1008A0006AE040EC51E00E94A10E4091090184E110
:1008B0006BE050E00E94FA0D20C082E062E047E861
:1008C00050E00E94A10E82E065E04CE151E00E9400
:1008D000A10EE199FECF88E190E09FBB8EBBE09A2C
:1008E0008DB38093C803E199FECF8AE190E09FBB6E
:1008F0008EBBE09A8DB3809309019091CD03892F2F
:1009000081708093C301892F88708093C401892FDF
:1009100080728093C50194709093C6011F910F91CE
:1009200008951F93809192018823E1F31092920120
:10093000809192018823E1F31092920183E666E7A9
:1009400040E00E948E1110E00DC08091970181302F
:1009500011F40E94490F80919201813019F4109294
:10096000920111E08091BD01882311F4112369F3F4
:10097000112309F054C082E062E045EC51E00E948E
:10098000A10E82E064E041EE51E00E94A10E82E0FF
:1009900066E040EF51E00E94A10E8091BC018130E1
:1009A00031F48EE064E04FEF51E00E94A10E80919F
:1009B000BC01823031F48EE064E043E052E00E94FA
:1009C000A10E8091BC01843031F48EE064E047E0F8
:1009D00052E00E94A10E409183038EE066E050E059
:1009E0000E94FA0D4091840380E166E050E00E948D
:1009F000FA0D4091850383E166E050E00E94FA0D14
:100A00002091BC01E199FECF89E190E09FBB8EBBB4
:100A10002DBB0FB6F894E29AE19A0FBE0AC0E19995
:100A2000FECF89E190E09FBB8EBBE09A8DB38093AF
:100A3000BC011F9108950E941F0383E66FE644E600
:100A40000E948E1180E06CE40E94D102109292010B
:100A5000809192018823E1F387E062E040E750E073
:100A60000E94A10E0E945D06109292018091920157
:100A70008823E1F310929201809192018823E1F39F
:100A800010929201809192018823E1F310929201D9
:100A9000809192018823E1F310929201809192015A
:100AA0008823E1F31092920184E064E00E94D10275
:100AB00080E06CE40E94D10280919901882319F4AE
:100AC0000E9491041CC082E062E04EE751E00E9467
:100AD000A10E82E064E044E951E00E94A10E82E0B0
:100AE00066E041EA51E00E94A10EE199FECF89E162
:100AF00090E09FBB8EBBE09A8DB38093BC01809148
:100B000092018823E1F3109292018091920188234F
:100B1000E1F31092920184E064E00E94D10280E04F
:100B20006CE40E94D10280919901882319F40E94FB
:100B3000360326C082E062E04EE351E00E94A10E3F
:100B400082E064E045E551E00E94A10E82E066E0AB
:100B500042E651E00E94A10EE199FECF88E190E0CB
:100B60009FBB8EBBE09A8DB38093C001E199FECF0D
:100B70008AE190E09FBB8EBBE09A8DB38093090120
:100B80008091BC01823029F483E66FE64AE00E943E
:100B90008E118091BC01813029F482E664E64AE03E
:100BA0000E948E11809192018823E1F310929201AC
:100BB000809192018823E1F3109292018091920139
:100BC0008823E1F310929201809192018823E1F34E
:100BD00010929201809192018823E1F31092920188
:100BE00084E064E00E94D102089582E083BF82E441
:100BF0008EBD8AE089BF08951F920F920FB60F92A3
:100C000011248F939F93809196018F5F809396011B
:100C100080919601883449F591E090939501109266
:100C200096018091E9038F5F8093E9038091E90346
:100C3000843631F41092E9039093920190939301DA
:100C40008091E903823319F481E0809393018091CC
:100C5000E8038F5F8093E8038091E8038A3029F4EA
:100C60001092E80381E0809394019F918F910F90FF
:100C70000FBE0F901F901895982F80538A3010F058
:100C800020E005C0903311F42AE001C0282F892FFD
:100C900081548A3110F4292F2653892F81568A31A5
:100CA00010F4292F2C539D3211F429E403C09E32F5
:100CB00009F421E4822F0895089585E060E00E9400
:100CC000D10286E063E80E94D10287E060E90E94D9
:100CD000D10285E060E00E94D10286E064E80E94D3
:100CE000D10287E061E90E94D10285E060E00E94C4
:100CF000D10286E065E80E94D10287E062E90E94A5
:100D0000D10285E060E00E94D10286E066E80E94A0
:100D1000D10287E063E90E94D10285E060E00E9491
:100D2000D10286E067E80E94D10287E064E90E9470
:100D3000D10285E060E00E94D10286E068E80E946E
:100D4000D10287E065E90E94D10285E060E00E945F
:100D5000D10286E069E80E94D10287E066E90E943C
:100D6000D10285E060E00E94D10286E06AE80E943C
:100D7000D10287E067E90E94D10285E060E00E942D
:100D8000D10286E061EA0E94D10287E068E90E9410
:100D9000D10285E060E00E94D10286E062EA0E9412
:100DA000D10287E069E90E94D10285E060E00E94FB
:100DB000D10286E063EA0E94D10287E06AE90E94DC
:100DC000D10285E060E00E94D10286E064EA0E94E0
:100DD000D10287E06BE90E94D10285E060E00E94C9
:100DE000D10286E065EA0E94D10287E06CE90E94A8
:100DF000D10285E060E00E94D10286E066EA0E94AE
:100E0000D10287E06DE90E94D10285E060E00E9496
:100E1000D10286E067EA0E94D10287E06EE90E9473
:100E2000D10285E060E00E94D10286E068EA0E947B
:100E3000D10287E06FE90E94D10285E060E00E9464
:100E4000D10286E06FEB0E94D10287E060EA0E9447
:100E5000D10285E060E00E94D10286E060EC0E9451
:100E6000D10287E061EA0E94D10285E060E00E9441
:100E7000D10286E061EC0E94D10287E062EA0E9422
:100E8000D10285E060E00E94D10286E062EC0E941F
:100E9000D10287E063EA0E94D10285E060E00E940F
:100EA000D10286E063EC0E94D10287E064EA0E94EE
:100EB000D10285E060E00E94D10286E064EC0E94ED
:100EC000D10287E065EA0E94D10285E060E00E94DD
:100ED000D10286E065EC0E94D10287E066EA0E94BA
:100EE000D10285E060E00E94D10286E066EC0E94BB
:100EF000D10287E067EA0E94D10285E060E00E94AB
:100F0000D10286E06DED0E94D10287E068EA0E947E
:100F1000D10285E060E00E94D10286E06EED0E9481
:100F2000D10287E069EA0E94D10285E060E00E9478
:100F3000D10286E06FED0E94D10287E06AEA0E944A
:100F4000D10285E060E00E94D10286E060EE0E945E
:100F5000D10287E06BEA0E94D10285E060E00E9446
:100F6000D10286E061EE0E94D10287E06CEA0E9425
:100F7000D10285E060E00E94D10286E062EE0E942C
:100F8000D10287E06DEA0E94D10285E060E00E9414
:100F9000D10286E063EE0E94D10287E06EEA0E94F1
:100FA000D10285E060E00E94D10286E064EE0E94FA
:100FB000D10287E06FEA0E94D10285E060E00E94E2
:100FC000D10286E06BEF0E94D10287E060EB0E94C5
:100FD000D10285E060E00E94D10286E06CEF0E94C1
:100FE000D10287E061EB0E94D10285E060E00E94BF
:100FF000D10286E06DEF0E94D10287E062EB0E9491
:10100000D10285E060E00E94D10286E06EEF0E948E
:10101000D10287E063EB0E94D10285E060E00E948C
:10102000D10286E06FEF0E94D10287E064EB0E945C
:10103000D10285E061E00E94D10286E060E00E947A
:10104000D10287E065EB0E94D10285E061E00E9459
:10105000D10286E061E00E94D10287E066EB0E9447
:10106000D1020895BF92CF92DF92EF92FF920F9339
:101070001F93CF93DF937C01B62E8C0145E0C42EE5
:10108000D12CC80ED91E862F90E0EC01CC0FDD1FAD
:10109000C80FD91FCA5EDE4F0EC085E0612F0E94C7
:1010A000D10286E0602F0E94D10287E068810E9411
:1010B000D1020F5F1F4F0C151D0578F38701065FE6
:1010C0001F4F8FE090E0E80EF91E8B2D90E0EC01B1
:1010D000CC0FDD1FC80FD91FCA5EDE4F0EC085E0E2
:1010E000612F0E94D10286E0602F0E94D10287E02A
:1010F00068810E94D1020F5F1F4F0E151F0578F304
:10110000DF91CF911F910F91FF90EF90DF90CF90E3
:10111000BF900895EF92FF920F931F93CF93DF93A9
:101120008C01EC0155E0E52EF12CE80EF91E0DC006
:1011300085E06D2F0E94D10286E06C2F0E94D102C3
:1011400087E060E00E94D1022196CE15DF0580F392
:10115000E8012A96015F1F4F0DC085E06D2F0E94A8
:10116000D10286E06C2F0E94D10287E060E00E94ED
:10117000D1022196C017D10780F3DF91CF911F9143
:101180000F91FF90EF9008951F93CF93DF93C0913D
:101190004702D0914802D7FD12C0CE016AE070E04C
:1011A0000E94771C182F16952091040130E0CE0183
:1011B0006AE070E00E94771C261B310918C0EE27F8
:1011C000FF27EC1BFD0BCF016AE070E00E94771C4B
:1011D000182F16951C5F2091040130E02F5F3F4FC0
:1011E000CF016AE070E00E94771C260F311DE901F3
:1011F00075E0CC0FDD1F7A95E1F7220F331FC21B7C
:10120000D30B27968091120190911301C817D9072B
:1012100039F080911201909113010E948A0804C054
:101220008091C901811721F0CE01612F0E943208FF
:101230001093C901D0931301C0931201DF91CF9194
:101240001F910895CF92DF92EF92FF920F931F9319
:10125000CF93DF938C01E62E85E0612F0E94D102AF
:1012600086E0602F0E94D102CE2CDD2484E391E041
:10127000C80ED91E87E0F60160810E94D102EEE11E
:10128000EE2EF12CE00EF11E85E06F2D0E94D102B2
:1012900086E06E2D0E94D10287E0F60160810E94F7
:1012A000D102E801CC54DF4F025F1E4F85E06D2F65
:1012B0000E94D10286E06C2F0E94D10287E0F601E5
:1012C00060810E94D1026E96C017D10779F7DF9135
:1012D000CF911F910F91FF90EF90DF90CF900895E5
:1012E000EF92FF920F931F93CF93DF937C0185E0E2
:1012F0006F2D0E94D10286E06E2D0E94D10287E000
:1013000060E00E94D1028701025E1F4F85E0612FDD
:101310000E94D10286E0602F0E94D10287E060E047
:101320000E94D102E701CC54DF4F8701025F1E4FBC
:1013300085E06D2F0E94D10286E06C2F0E94D102C1
:1013400087E060E00E94D1026E96C017D10781F756
:10135000DF91CF911F910F91FF90EF9008951F9310
:10136000CF93DF93E0914502F0914602F7FD14C060
:10137000CF016AE070E00E94771C182F16951C5F61
:1013800080910501C82FD0E0CF016AE070E00E9493
:10139000771CC61BD10917C0222733272E1B3F0BF2
:1013A000C9016AE070E00E94771C182F16958091A1
:1013B0000501C82FD0E02196C9016AE070E00E94C3
:1013C000771CC60FD11D8091140190911501C8178B
:1013D000D90739F080911401909115010E9470098C
:1013E00004C08091CA01811721F0CE01612F0E94B3
:1013F00022091093CA01D0931501C0931401DF9103
:10140000CF911F91089585E060E00E94D10286E0AF
:101410006FEC0E94D10287E06CE80E94D10285E067
:1014200061E00E94D10286E06BE00E94D10287E079
:101430006DE80E94D1020895EF92FF920F931F93DF
:10144000CF93DF937A019EE1699FB0011124680F69
:10145000711D8B01020F111D1092EA03EB0115C0E3
:1014600085E06D2F0E94D10286E06C2F0E94D10290
:101470008091EA03F701E80FF11D60818F5F80938F
:10148000EA0387E00E94D1022196C017D10740F3FA
:10149000DF91CF911F910F91FF90EF900895609190
:1014A000030181E04DE051E025E00E941C0A08950F
:1014B000DF93CF9300D000D0CDB7DEB7F894309152
:1014C0004D027894832F6AE00E944A1C282F0E94C4
:1014D0004A1C482F822F0E944A1C292F832F0E94CA
:1014E0004A1C992319F48AE08C8301C09C8322232F
:1014F00019F48AE08A8301C02A83498385E48B83B7
:1015000083E061E0AE014F5F5F4F24E00E941C0A60
:101510000F900F900F900F90CF91DF910895DF9370
:10152000CF9300D000D0CDB7DEB780E289839BE0B7
:101530009A8381E38B839C8381E061E0AE014F5FFE
:101540005F4F21E00E941C0A80919B01813079F459
:1015500062E0AE014E5F5F4F21E00E941C0A81E015
:1015600063E0AE014D5F5F4F22E00E941C0A0F90C6
:101570000F900F900F90CF91DF910895DF93CF934D
:1015800000D000D00F92CDB7DEB7DE011196E1E4B6
:10159000F1E085E001900D928150E1F76091040146
:1015A0008CE0AE014F5F5F4F25E00E941C0A0F9058
:1015B0000F900F900F900F90CF91DF91089580E0E2
:1015C0006CE40E94D10208958091570390915803D2
:1015D000843B910554F08091D80390E0209155030D
:1015E000309156038217930744F08091CB018823F2
:1015F00071F481E08093CB0108958091CB0118169E
:1016000024F480E06CE40E94D1021092CB01089592
:1016100080E062E40E94D10208958F929F92AF927F
:10162000BF92CF92DF92EF92FF920F931F93DF93BF
:10163000CF93CDB7DEB72F970FB6F894DEBF0FBEAE
:10164000CDBFFE013B9685E0DF011D928A95E9F74B
:101650008091490290914A026EE170E00E94771CED
:10166000CB01019797FF02C080E090E08E010F5FF1
:101670001F4FB8014AE050E00E94111CF801019090
:101680000020E9F73197FE2EF01A80E0CF2CDD2400
:10169000C7FCD094F6E08F2E912C8C0E9D1E580125
:1016A0000BC0F501E00FF11F80810E943C06080D80
:1016B000191DF80180838E2D082F10E0E82EE39489
:1016C0000C151D0574F38093EA0385E169E0AE0112
:1016D000455F5F4F25E00E941C0A89E18F1969E090
:1016E000A4012F2D0E941C0A2F960FB6F894DEBF7E
:1016F0000FBECDBFCF91DF911F910F91FF90EF9063
:10170000DF90CF90BF90AF909F908F9008958F9271
:101710009F92AF92BF92CF92DF92EF92FF920F9380
:101720001F93DF93CF93CDB7DEB72E970FB6F89404
:10173000DEBF0FBECDBF19821A821B821C82809130
:10174000B0019091B1018E010B5F1F4FB8014AE0CB
:1017500050E00E94111CF80101900020E9F7319738
:10176000FE2EF01A80E0CF2CDD24C7FCD094AAE036
:101770008A2E912C8C0E9D1E58010BC0F501E00F96
:10178000F11F80810E943C06080D191DF80180831D
:101790008E2D082F10E0E82EE3940C151D0574F330
:1017A0008093EA0385E166E0AE014F5F5F4F24E07E
:1017B0000E941C0A89E18F1966E0A4012F2D0E9466
:1017C0001C0A8091B0019091B1011816190664F4B9
:1017D00085E060E00E94D10286E062EC0E94D102C6
:1017E00087E06CE80E94D1028091B0019091B10134
:1017F00097FF0CC085E060E00E94D10286E062ECB9
:101800000E94D10287E06DE80E94D1028091B00170
:101810009091B101892B61F485E060E00E94D102D2
:1018200086E062EC0E94D10287E060E00E94D10273
:101830002E960FB6F894DEBF0FBECDBFCF91DF91CD
:101840001F910F91FF90EF90DF90CF90BF90AF90DE
:101850009F908F9008958F929F92AF92BF92CF9258
:10186000DF92EF92FF920F931F93DF93CF93CDB749
:10187000DEB72B970FB6F894DEBF0FBECDBFDE01EB
:101880001196EEE3F1E083E001900D928150E1F7D3
:101890008E010C5F1F4F8091530390915403B80148
:1018A0004AE050E00E94111CF80101900020E9F785
:1018B0003197FE2EF01A80E0CF2CDD24C7FCD094A7
:1018C000B8E08B2E912C8C0E9D1E58010BC0F5019B
:1018D000E00FF11F80810E943C06080D191DF801E0
:1018E00080838E2D082F10E0E82EE3940C151D0543
:1018F00074F38093EA038DE06EE0AE014F5F5F4FBB
:1019000023E00E941C0A80E18F196EE0A4012F2DB4
:101910000E941C0A2B960FB6F894DEBF0FBECDBFF7
:10192000CF91DF911F910F91FF90EF90DF90CF90BB
:10193000BF90AF909F908F9008958F929F92AF929B
:10194000BF92DF92EF92FF920F931F93DF93CF939B
:10195000CDB7DEB728970FB6F894DEBF0FBECDBF68
:1019600019828AE08A838091A2019091A3018E015D
:101970000D5F1F4FB8014AE050E00E94111CF801B2
:1019800001900020E9F73197E01B80E0EE2EFF2464
:10199000E7FCF094480106E0A02EB12CAC0EBD1E71
:1019A0000BC0F401E00FF11F80810E943C060A0D7C
:1019B0001B1DF80180838D2D082F10E0D82ED394A5
:1019C0000E151F0574F38093EA038091A201909194
:1019D000A3018E010A5F1F4F0A977CF460910301F7
:1019E00081E0AE014F5F5F4F21E00E941C0A6091D1
:1019F000030182E0A80121E005C06091030181E0BC
:101A0000A80122E00E941C0A8091A4019091A501E6
:101A10008E010D5F1F4FB8014AE050E00E94111C7B
:101A2000F80101900020E9F73197E01B80E0EE2EED
:101A3000FF24E7FCF094480116E0A12EB12CAC0E77
:101A4000BD1E0BC0F401E00FF11F80810E943C0617
:101A50000A0D1B1DF80180838D2D082F10E0D82E54
:101A6000D3940E151F0574F38093EA038091A401AB
:101A70009091A5018E010A5F1F4F0A977CF4609137
:101A8000030184E0AE014E5F5F4F21E00E941C0A1B
:101A90006091030185E0A80121E005C06091030188
:101AA00084E0A80122E00E941C0A28960FB6F89450
:101AB000DEBF0FBECDBFCF91DF911F910F91FF9081
:101AC000EF90DF90BF90AF909F908F9008950F930D
:101AD0001F93DF93CF93CDB7DEB72A970FB6F89455
:101AE000DEBF0FBECDBF8E010F5F1F4FB8014AE0B2
:101AF00050E00E94111CF80101900020E9F7319795
:101B0000E01B20E0FF27E7FDF095322F3F5F822F9B
:101B100090E08E179F0714F4232FF7CF2093EA034A
:101B20002A960FB6F894DEBF0FBECDBFCF91DF91DE
:101B30001F910F910895AF92BF92CF92DF92EF92D3
:101B4000FF920F931F93DF93CF93CDB7DEB76E97BE
:101B50000FB6F894DEBF0FBECDBFB82EA62ED42E82
:101B6000A42FB52FFD0101900020E9F73197CE2E6B
:101B7000C41A7E010894E11CF11C242F352FC901E1
:101B80008C0108C0F80181918F010E943C06F70189
:101B900081937F01802F8D198C15A0F38B2D6A2DD9
:101BA000AE014F5F5F4F2C2D0E941C0A6E960FB640
:101BB000F894DEBF0FBECDBFCF91DF911F910F9183
:101BC000FF90EF90DF90CF90BF90AF9008958091FD
:101BD0009A01813071F4609106012091E101309108
:101BE000E201369527958EE0821B43EE51E00E947C
:101BF0009B0D0895EF92FF920F931F93DF93CF9366
:101C0000CDB7DEB764970FB6F894DEBF0FBECDBF79
:101C1000F82EE62ECA018E010F5F1F4FB8014AE071
:101C200050E00E94111C8F2D6E2DA8010E949B0D6B
:101C300064960FB6F894DEBF0FBECDBFCF91DF9193
:101C40001F910F91FF90EF900895EF92FF920F93E5
:101C50001F93DF93CF93CDB7DEB72A970FB6F894D3
:101C6000DEBF0FBECDBF20919203822F6AE00E949B
:101C7000561C382F822F6AE00E94561C85E48F8301
:101C800080919303882309F48AE08887992319F4C3
:101C90008AE08E8301C09E833D8319821A821B8253
:101CA0001C8283E062E0AE014B5F5F4F24E00E9444
:101CB0001C0A80919603909197038952934234F0C5
:101CC00088E293E290939703809396038091960322
:101CD0009091970397FF04C0109297031092960378
:101CE0008E010B5F1F4F8091960390919703B8016F
:101CF0004AE050E00E94111CF80101900020E9F731
:101D00007F010894E108F108E01AF10A83E063E03A
:101D1000AE014F5F5F4F24E00E941C0A87E08E19DE
:101D200063E0A8010E949B0D2A960FB6F894DEBFCF
:101D30000FBECDBFCF91DF911F910F91FF90EF901C
:101D40000895BF92CF92DF92EF92FF920F931F936D
:101D5000DF93CF93CDB7DEB764970FB6F894DEBFAD
:101D60000FBECDBFC82EB62EFA017E010894E11C2D
:101D7000F11C04C0AE0DBF1D9C9331968E2F841BA9
:101D80009491A82FB0E09923A9F7AE0DBF1D1C9226
:101D9000F70101900020E9F73197DE2EDE18870168
:101DA00007C0F80180810E943C06F80181938F01F1
:101DB000802F8E198D15A8F38C2D6B2DAE014F5FE2
:101DC0005F4F2D2D0E941C0A64960FB6F894DEBF5B
:101DD0000FBECDBFCF91DF911F910F91FF90EF907C
:101DE000DF90CF90BF9008951F93CF93DF93EC01C6
:101DF000A3E0B0E047C0FD01E758FD4F8081FD0141
:101E0000E658FD4F2081422F50E04D535040FD01D8
:101E1000E558FD4F7081FD01E458FD4F10819A0196
:101E2000F4E035952795FA95E1F790E0CD97880F86
:101E3000991F880F991F282B392B2883613029F18E
:101E4000E72FF0E0FD9734E0440F551F3A95E1F796
:101E50005070CF019595879595958795482B592B6F
:101E60004983623091F01496635086E0EE0FFF1FB5
:101E70008A95E1F7F070812F90E0CD97E82BF92B50
:101E8000EA832396662309F0B6CFDF91CF911F91A5
:101E9000089580917B028635B1F480917A02815653
:101EA0008093BC018091BC01843018F084E0809361
:101EB000BC0183E893E06AE043E02AE00E94F40E6C
:101EC00081E08093BD011092970108951F931091B6
:101ED000BC01123009F474C0143009F4C9C01130C7
:101EE00009F089C180917B02813581F48FEB93E009
:101EF00062E343E02DE20E94F40E8091BF0390E084
:101F00009093BF018093BE011093C20180917B0228
:101F1000843409F070C181E493E061E443E021E49A
:101F20000E94F40E8091570390915803843B9105D1
:101F30003CF480919C01813051F410929C0107C0C7
:101F400080919C01882319F481E080939C01809109
:101F500043039091440365EF7FEF0E94771C6E5F0F
:101F60007F4F7093480260934702809145039091A0
:101F700046036BE070E00E94771C6A5F7F4F7093AE
:101F800046026093450280914D0390914E039093D9
:101F90004A02809349028091550380934D028091BB
:101FA0002C0290912D0290934C0280934B028091D1
:101FB0005303909154039093500280934F021BC19E
:101FC00080917B028F34A9F0813509F014C18FEB29
:101FD00093E062E343E02DE20E94F40E8091BF03A0
:101FE00090E09093BF018093BE0181E08093C20195
:101FF00002C187EF91E060E543E02DE20E94F40E1C
:1020000080913702992787FD909502969093480218
:102010008093470280913802992787FD9095069614
:10202000909346028093450280912A0290912B0260
:1020300090934A02809349028091300280934D022E
:1020400080912C0290912D0290934C0280934B0230
:1020500080913502909136029093500280934F0206
:10206000809129028093510281E08093C101C3C015
:1020700080917B02843409F05AC081E493E061E4EA
:1020800043E021E40E94F40E80915703909158039D
:10209000843B910554F480919C01813031F410927D
:1020A0009C01F8940E940F117894809157039091AD
:1020B0005803843B91057CF080919C01882359F45E
:1020C00081E080939C01F89480919901882311F418
:1020D0000E94FF107894809143039091440366E13D
:1020E00070E00E94771C6E5F7F4F70934802609390
:1020F0004702809145039091460366E170E00E949B
:10210000771C6A5F7F4F709346026093450280910F
:102110004D0390914E0390934A028093490280911F
:102120005303909154039093500280934F028091F7
:102130007B028C3481F481E090E09093BF01809326
:10214000BE0181E08093C20180EC93E069E143E04D
:102150002DE20E94F40E80917B028D3481F482E0A6
:1021600090E09093BF018093BE0181E08093C20113
:1021700080EC93E069E143E02DE20E94F40E80914F
:102180007B028E3481F483E090E09093BF018093D2
:10219000BE0181E08093C20180EC93E069E143E0FD
:1021A0002DE20E94F40E80917B028F3481F484E052
:1021B00090E09093BF018093BE0181E08093C201C3
:1021C00080EC93E069E143E02DE20E94F40E8091FF
:1021D0007B02803581F485E090E09093BF0180938D
:1021E000BE0181E08093C20180EC93E069E143E0AD
:1021F0002DE20E94F40E109297011F91089582E241
:1022000089B910BC80B91CBE909A28E92AB996E811
:1022100090BD82EC8BB921B99CBF82B9089582E24E
:1022200089B910BC80B91CBE88E98AB926E820BDEE
:1022300092EC9BB980E981B92CBF92B90895DF93E4
:10224000CF93CDB7DEB72C970FB6F894DEBF0FBE95
:10225000CDBF83E2898383E68A8385E78B838DE321
:102260008C838D838E838F83DE011196FD0120E0A8
:1022700030E0AE01485F5F4F8191280F311DE417B8
:10228000F507D1F7C9019F7046E0959587954A9566
:10229000E1F7835C88872F733070822F835C898796
:1022A0008DE08A879E01255F3F4F8C91159BFECF65
:1022B00083B91196A217B307C1F72C960FB6F894FD
:1022C000DEBF0FBECDBFCF91DF910895DF93CF93D7
:1022D000CDB7DEB72C970FB6F894DEBF0FBECDBFDB
:1022E0008BE189838A8385E58B838AEA8C831D82CF
:1022F000FE0131969E012A5F3F4F8081159BFECFE4
:1023000083B93196E217F307C1F72C960FB6F8940C
:10231000DEBF0FBECDBFCF91DF910895DF93CF9386
:10232000CDB7DEB72A970FB6F894DEBF0FBECDBF8C
:1023300093E299838A836B83842F86958695835C49
:102340008C8350E04370507064E0440F551F6A95D1
:10235000E1F7435C4D838DE38E838F83DE0111961D
:10236000FD0120E030E0AE01485F5F4F8191280F12
:10237000311DE417F507D1F7C9019F7056E0959517
:1023800087955A95E1F7835C88872F733070822F89
:10239000835C89878DE08A879E01255F3F4F8C9102
:1023A000159BFECF83B91196A217B307C1F72A96E2
:1023B0000FB6F894DEBF0FBECDBFCF91DF91089569
:1023C0005D9BFECF8DE68CB95D9BFECF8FE68CB911
:1023D0005D9BFECF89E68CB95D9BFECF8EE68CB906
:1023E0005D9BFECF8DE08CB95D9BFECF8EE38CB9FB
:1023F0000895982F9F7082958F708A3010F4805DB9
:1024000001C0895C5D9BFECF8CB99A3018F4892F8E
:10241000805D02C0892F895C5D9BFECF8CB90895D9
:102420008A3010F4805D01C0895C5D9BFECF8CB961
:102430000895159BFECF83B908955D9BFECF8CB99F
:102440000895662359F020E0FC01E20FF11DE081C0
:102450005D9BFECFECB92F5F6217B0F708955D9BCF
:10246000FECF8EE38CB908951F920F920FB60F9294
:1024700011242F933F938F939F93AF93BF93EF9329
:10248000FF932CB12093EB0385B398E0892785BB9C
:102490005D9BFECF2CB92D3059F08091BE03E82F03
:1024A000F0E0E856FC4F20838F5F8093BE035FC04F
:1024B000E091BE03F0E0E856FC4F20831092B90192
:1024C0001092BA011092BB0130E020E090E045C0CC
:1024D0002130B9F0213018F02230F1F528C0A32FB7
:1024E000B0E0A856BC4F8C91803211F421E033C08B
:1024F000E92FF0E08C91EA54FC4F80839093B9016E
:102500000FC0A32FB0E0A856BC4F8C91E92FF0E08C
:10251000803241F08C91E459FD4F80839093BA0151
:102520009F5F1AC0E459FD4F108222E014C0A32F10
:10253000B0E0A856BC4F8C91E92FF0E08D3039F017
:102540008C91ED5AFD4F80839093BB01E9CFED5AFA
:10255000FD4F108223E090E03F5F8091BE03831720
:1025600008F0B6CF81E08093B8011092BE03FF91CE
:10257000EF91BF91AF919F918F913F912F910F90CC
:102580000FBE0F901F9018951F920F920FB60F92CB
:1025900011248F939F93EF93FF9393B19093EC0348
:1025A0009D3081F48091CC01813061F4AB98109220
:1025B000CC0180939701E0918E03F0E0E758FD4F46
:1025C00090832DC08091CC01882319F0813039F59A
:1025D00014C0933241F480919701882321F481E063
:1025E0008093CC01AB9A10928E0380918E03E82FDA
:1025F000F0E0E758FD4F90830CC0E0918E03F0E0CF
:10260000E758FD4F908380918E03873C30F4809192
:102610008E038F5F80938E0302C01092CC01FF91D6
:10262000EF919F918F910F900FBE0F901F90189573
:1026300085B392E0892785BB089590919F019130E1
:1026400019F485B3892785BB08951F920F920FB6A1
:102650000F9211242F933F935F936F937F938F93E8
:102660009F93AF93BF938091CE019091CF01892B1F
:1026700081F484B595B59093D5018093D4018EB53E
:102680008F7B8EBD81E090E09093CF018093CE014F
:102690003AC084B595B59093D3018093D2012EB5FD
:1026A00020642EBD2091D4013091D5011092CF012C
:1026B0001092CE01821B930B865698406CE271E01B
:1026C0000E94631C7093D1016093D0016730710543
:1026D00034F086E090E09093D1018093D001209176
:1026E000D0013091D10180910201992787FD909509
:1026F0002817390741F0263031052CF420930201C8
:1027000081E08093A601BF91AF919F918F917F91BE
:102710006F915F913F912F910F900FBE0F901F907F
:1027200018958091490290914A029093A901809353
:10273000A8018091A8019091A9012091AA0130914E
:10274000AB01821B930B9093AD018093AC01809100
:10275000A8019091A9019093AB018093AA014091A7
:10276000B4015091B5018091AC019091AD01E3E0CD
:10277000880F991FEA95E1F79A0173E0220F331F42
:102780007A95E1F7241B350B820F931F68E070E008
:102790000E94771C7093B5016093B4012091B6013B
:1027A0003091B7014091B4015091B501C90163E086
:1027B000880F991F6A95E1F7821B930B840F951F71
:1027C00068E070E00E94771C7093B7016093B601D7
:1027D0008091B6019091B7019093B1018093B001BF
:1027E0000E94870B0895609104018BE14EE451E053
:1027F0000E949B0D80913B0281FF07C06091040104
:102800008BE141E551E00E949B0D80913B0282FFEC
:1028100007C0609104018BE144E551E00E949B0DEB
:102820000895DF93CF930F92CDB7DEB78091250245
:102830009091260221E0823592071CF080EC89837A
:1028400007C04E966DE270E00E94771C6054698369
:10285000609104018EE0AE014F5F5F4F21E00E9466
:102860001C0A0F90CF91DF9108958AE161E047E55E
:1028700051E022E00E941C0A0895DF93CF9300D01C
:1028800000D0CDB7DEB719821A821B821C826091FC
:102890000301615085E1AE014F5F5F4F24E00E946C
:1028A0001C0A609103016150409112025091130281
:1028B00085E10E94FA0D0F900F900F900F90CF912D
:1028C000DF910895DF93CF9300D00F92CDB7DEB79D
:1028D000DE011196E9E5F1E083E001900D9281506F
:1028E000E1F7609104016F5F8EE0AE014F5F5F4FD3
:1028F00023E00E941C0A209104012F5F8091230293
:10290000909124026AE070E00E94771CAB018EE097
:10291000622F0E94FA0D0F900F900F90CF91DF91D0
:1029200008958F929F92BF92CF92DF92EF92FF9283
:102930000F931F93DF93CF93CDB7DEB72B970FB6CF
:10294000F894DEBF0FBECDBFDE011196ECE5F1E0DD
:1029500083E001900D928150E1F7809151028E0148
:102960000C5F1F4F90E0B8014AE050E00E94111C3C
:10297000F80101900020E9F73197BE2EB01AEE243D
:10298000FF24CB2CDD24C7FCD09488E0882E912C2A
:102990008C0E9D1E0DC0F801EE0DFF1D80810E9462
:1029A0003C06F401EE0DFF1D80830894E11CF11C30
:1029B000EC14FD0484F388E161E0AE014F5F5F4FEA
:1029C00023E00E941C0A8BE18B1961E0A4012B2DEE
:1029D0000E941C0A2B960FB6F894DEBF0FBECDBF27
:1029E000CF91DF911F910F91FF90EF90DF90CF90EB
:1029F000BF909F908F9008958F929F92BF92CF9299
:102A0000DF92EF92FF920F931F93DF93CF93CDB797
:102A1000DEB76A970FB6F894DEBF0FBECDBFFE01DA
:102A2000319686E0DF011D928A95E9F72091310207
:102A300030913202C90143E0880F991F4A95E1F7AE
:102A4000820F931F6AEF70E00E94631CCB018E011E
:102A5000095F1F4FB8014AE050E00E94111CF801C5
:102A600001900020E9F73197BE2EB01AEE24FF2422
:102A7000CB2CDD24C7FCD09491E1892E912C8C0EB7
:102A80009D1E0DC0F801EE0DFF1D80810E943C06C9
:102A9000F401EE0DFF1D80830894E11CF11CEC1481
:102AA000FD0484F36091030185E1AE014F5F5F4F48
:102AB00026E00E941C0A609103018BE18B19A4019E
:102AC0002B2D0E941C0A6A960FB6F894DEBF0FBE2B
:102AD000CDBFCF91DF911F910F91FF90EF90DF90CD
:102AE000CF90BF909F908F90089583E66FE644E665
:102AF0000E948E11F89428E088E190E00FB6F894D7
:102B0000A89581BD0FBE21BDFFCF1F939D998AC19E
:102B10008091D6018F5F8093D60111E01093D80188
:102B20008091D601853009F081C18091DA01882336
:102B300009F08CC01093DA011092DB0184E064E0AC
:102B40000E94D10283E061E043EE51E00E949B0DC0
:102B500083E063E042E152E00E94A10E84E068E07D
:102B60000E94D10283E065E04BE152E00E94A10E99
:102B700080910001813029F484E165E047E452E06E
:102B800004C084E165E04AE452E00E94A10E84E0C2
:102B900060E00E94D10283E066E04FE152E00E94D3
:102BA000A10E80919901813029F484E166E047E427
:102BB00052E004C084E166E04AE452E00E94A10EC3
:102BC00083E067E045E252E00E94A10E80919A0105
:102BD000813029F484E167E047E452E004C084E1F5
:102BE00067E04AE452E00E94A10E83E068E04DE213
:102BF00052E00E94A10E8091A701813029F484E166
:102C000068E047E452E004C084E168E04AE452E04E
:102C10000E94A10E83E069E048E352E00E94A10E09
:102C200080919B01813029F484E169E047E452E01E
:102C300004C084E169E04AE452E00E94A10E83E00E
:102C40006BE042E452E00E94A10EEEC08091DB01F5
:102C5000882349F584E068E00E94D1028091000158
:102C6000882339F41093000184E165E047E452E0E1
:102C700006C01092000184E165E04AE452E00E943F
:102C8000A10E20910001E199FECF81E090E09FBB71
:102C90008EBB2DBB0FB6F894E29AE19A0FBE84E08A
:102CA00060E00E94D1021091DB01113049F584E00F
:102CB00068E00E94D10280919901882339F4109331
:102CC000990184E166E047E452E006C01092990160
:102CD00084E166E04AE452E00E94A10E209199014D
:102CE000E199FECF80E090E09FBB8EBB2DBB0FB67D
:102CF000F894E29AE19A0FBE84E060E00E94D1026B
:102D00008091DB01823051F584E068E00E94D102BD
:102D100080919A01882341F481E080939A0184E1B3
:102D200067E047E452E006C010929A0184E167E050
:102D30004AE452E00E94A10E20919A01E199FECF4F
:102D400082E090E09FBB8EBB2DBB0FB6F894E29A59
:102D5000E19A0FBE84E060E00E94D1028091DB0125
:102D6000833051F584E068E00E94D1028091A70190
:102D7000882341F481E08093A70184E168E047E47F
:102D800052E006C01092A70184E168E04AE452E0F4
:102D90000E94A10E2091A701E199FECF87E190E06A
:102DA0009FBB8EBB2DBB0FB6F894E29AE19A0FBE83
:102DB00084E060E00E94D1028091DB01843049F51B
:102DC00068E00E94D10280919B01882341F481E058
:102DD00080939B0184E169E047E452E006C01092D1
:102DE0009B0184E169E04AE452E00E94A10E209137
:102DF0009B01E199FECF8BE190E09FBB8EBB2DBB89
:102E00000FB6F894E29AE19A0FBE84E060E00E9467
:102E1000D1028091DB01853049F41092DA010E94E1
:102E2000751504C01092D6011092D8019C9913C157
:102E30009091DA01913009F014C19093D9018091F9
:102E4000D7018F5F8093D7012091D701253009F0FA
:102E500008C11092D7018091DB01823009F469C06A
:102E6000833030F4882371F0813009F0FAC035C026
:102E7000843009F4AAC0843008F486C0853009F093
:102E8000F0C0C3C09093DB0183E065E04BE152E00A
:102E90000E94A10E80910001813029F484E165E057
:102EA00047E452E004C084E165E04AE452E00E9455
:102EB000A10E84E068E00E94D10283E066E04FE169
:102EC00052E00E94A10E80919901813019F484E1B1
:102ED00066E0B3C084E166E0B5C082E08093DB01C8
:102EE00083E066E04FE152E00E94A10E80919901DB
:102EF000813029F484E166E047E452E004C084E1D3
:102F000066E04AE452E00E94A10E84E068E00E947C
:102F1000D10283E067E045E252E00E94A10E809179
:102F20009A01813019F484E167E087C084E167E0A9
:102F300089C083E08093DB0167E045E252E00E94B4
:102F4000A10E80919A01813029F484E167E047E481
:102F500052E004C084E167E04AE452E00E94A10E1E
:102F600084E068E00E94D10283E068E04DE252E034
:102F70000E94A10E8091A701813019F484E168E0DC
:102F80005CC084E168E05EC084E08093DB0183E0A4
:102F900068E04DE252E00E94A10E8091A7018130CD
:102FA00029F484E168E047E452E004C084E168E089
:102FB0004AE452E00E94A10E84E068E00E94D1023F
:102FC00083E069E048E352E03FC02093DB0183E007
:102FD00069E048E352E00E94A10E80919B0181309C
:102FE00029F484E169E047E452E004C084E169E047
:102FF0004AE452E00E94A10E84E068E00E94D102FF
:1030000083E06BE042E452E01FC01092DB0183E0FA
:103010006BE042E452E00E94A10E84E068E00E946E
:10302000D10283E065E04BE152E00E94A10E809165
:103030000001813029F484E165E047E452E004C0F6
:1030400084E165E04AE452E00E94A10E84E060E081
:103050000E94D10206C01092D7018091D8018091C0
:10306000D9011F910895813061F4E199FECF80E08C
:1030700090E09FBB8EBB6DBB0FB6F894E29AE19ACD
:103080000FBE0895DF93CF93CDB7DEB764970FB629
:10309000F894DEBF0FBECDBF20E0DE011196E199AE
:1030A000FECFE22FF0E0CF018D5F9F4F9FBB8EBB25
:1030B000E09A8DB3EA0FFB1F8083882311F02F5F06
:1030C000EECFFD0101900020E9F79F012150304033
:1030D0002A1B3B0B3093E2012093E10190E0AE010B
:1030E0004F5F5F4F09C0FD01ED51FE4FA40FB51FAB
:1030F0008C91808311829F5FA92FB0E0A217B30744
:1031000090F364960FB6F894DEBF0FBECDBFCF919B
:10311000DF910895DF93CF93CDB7DEB760970FB6F9
:10312000F894DEBF0FBECDBF80914F029091500248
:103130009093780280937702809177029091780241
:103140006FE070E00E94631CDE011596AD016A1B02
:103150009E01205F3F4FE62FEA0FF0E0E35BFD4F5B
:10316000E491ED93A217B307B1F7609107011982BB
:103170001A821B821C8289E02BE00E941C0A60914B
:1031800008018EE0AE014F5F5F4F24E00E941C0AF1
:103190006091080140917702509178028FE00E947F
:1031A000FA0D60960FB6F894DEBF0FBECDBFCF917B
:1031B000DF910895FF920F931F93DF93CF93CDB7C5
:1031C000DEB7E4970FB6F894DEBF0FBECDBFDE01C9
:1031D0001C96EFE5F1E087E001900D928150E1F758
:1031E000DE015396E6E6F1E089E001900D92815010
:1031F000E1F7DE019796EFE6F1E08EE001900D92A7
:103200008150E1F7DE011696EDE7F1E086E00190EE
:103210000D928150E1F7DE015C96E3E8F1E08BE08E
:1032200001900D928150E1F78091B6039091B70320
:10323000873409F066C0943409F063C080916C0251
:1032400090916D02813409F05CC09C3409F059C042
:10325000E199FECF81E090E09FBB8EBBE09A2DB359
:10326000211121E0022FE199FECF80E090E09FBB89
:103270008EBBE09A8DB3882311F0022F0260E19992
:10328000FECF82E090E09FBB8EBBE09A8DB38111B0
:103290000460E199FECF87E190E09FBB8EBBE09A8E
:1032A0008DB381110860E199FECF8BE190E09FBB67
:1032B0008EBBE09A8DB38111006183E20E941D12E2
:1032C000802F90E08E010F5F1F4FB8014AE050E061
:1032D0000E94111CF80101900020E9F73197E01BD2
:1032E000F10BC8016E2F0E9421128CE20E941D1268
:1032F00083EE91E06091E1010E9421128DE00E9435
:103300001D128091B6039091B703833509F0B6C0C2
:10331000943409F0B3C08CE692E00E94EC1BF82EC6
:1033200003EE11E0C80163E572E00E940A1CD801B7
:103330000D900020E9F71197A01BB10B80E011C0A0
:10334000F901ED51FE4FE081E199FECF2D5F3F4F36
:103350003FBB2EBBEDBB0FB6F894E29AE19A0FBECD
:103360008F5F282F30E02A173B0750F3E199FECFFB
:103370008F5F90E08D5F9F4F9FBB8EBB1DBA0FB6D6
:10338000F894E29AE19A0FBEB093E201A093E101B2
:103390002F2DF0FE09C0E199FECF81E090E09FBBA8
:1033A0008EBB81E08DBB07C0E199FECF81E090E04C
:1033B0009FBB8EBB1DBA0FB6F894E29AE19A0FBE7E
:1033C00021FF09C0E199FECF80E090E09FBB8EBB5A
:1033D00081E08DBB07C0E199FECF80E090E09FBB0C
:1033E0008EBB1DBA0FB6F894E29AE19A0FBE22FF87
:1033F00009C0E199FECF82E090E09FBB8EBB81E0E7
:103400008DBB07C0E199FECF82E090E09FBB8EBBF1
:103410001DBA0FB6F894E29AE19A0FBE23FF09C0D5
:10342000E199FECF87E190E09FBB8EBB81E08DBB31
:1034300007C0E199FECF87E190E09FBB8EBB1DBA2C
:103440000FB6F894E29AE19A0FBE24FF09C0E19901
:10345000FECF8BE190E09FBB8EBB81E08DBB07C0B0
:10346000E199FECF8BE190E09FBB8EBB1DBA0FB6FA
:10347000F894E29AE19A0FBE0E9475155091B60336
:103480006091B7034091B8038091B90320E030E028
:10349000803711F421E030E080E090E04C3611F408
:1034A00081E090E02823392380E0583609F481E058
:1034B00090E0653609F491E0892390E028233923D0
:1034C000232B79F0CE010C9666E00E942112CE01EA
:1034D000439668E00E942112CE0187966DE00E941B
:1034E00021125091B6036091B7034091B8038091C7
:1034F000B90320E030E0873711F421E030E080E0CC
:1035000090E04F3611F481E090E02823392380E0E9
:10351000533709F481E090E0683609F491E089239B
:1035200090E028233923232B19F180916C0290918C
:103530006D02893481F4943471F4CE01069665E00D
:103540000E94211283EE91E06091E1010E9421121C
:103550008DE00E941D1280916C0290916D02863761
:1035600039F4953629F4CE014C966CE00E94211274
:103570008091B6032091B7034091B80390E0833760
:1035800009F491E080E0253609F481E09823892F41
:1035900090E020E030E0443711F421E030E0822375
:1035A0009323892B09F442C080916C0290916D02A3
:1035B000893409F03BC0943409F038C020E01AC0C7
:1035C000FD01ED5AFD4FE081E199FECF822F90E0A1
:1035D0008D5F9F4F9FBB8EBBEDBB0FB6F894E29AF9
:1035E000E19A0FBEFD01ED5AFD4F8081AD51BE4FF6
:1035F0008C932F5F8091BB01A22FB0E0281700F3BE
:10360000E199FECFCD018D5F9F4F9FBB8EBB1DBA51
:103610000FB6F894E29AE19A0FBEE22FF0E0ED5176
:10362000FE4F1082B093E201A093E1015091B603E6
:103630006091B7034091B8038091B90320E030E076
:10364000853611F421E030E080E090E0433711F45A
:1036500081E090E02823392380E0523709F481E0AB
:1036600090E0653609F491E0892390E0282339231E
:10367000232B11F00E947515E4960FB6F894DEBF67
:103680000FBECDBFCF91DF911F910F91FF90089595
:103690001F920F920FB60F9211242F933F938F9387
:1036A0009F93EF93FF938091DD01882381F08091B8
:1036B000DD0190E00197E0919001F0919101E80F18
:1036C000F91F8FB1808381E08093DE0103C08FB149
:1036D0008093F2032091DD0180918E0130E09927E3
:1036E00087FD9095821793075CF084E080938F01AB
:1036F00081E08093DE018091DD018093F10308C0B9
:10370000929A1092DC0181E08093DF011092E00137
:103710008091DD018F5F8093DD01FF91EF919F919B
:103720008F913F912F910F900FBE0F901F90189582
:1037300082ED8DB90895813029F4613011F49298A9
:103740000895929A0895982F8091DC018823C9F4F6
:10375000913009F492989093DC0181E08093E0012C
:10376000913069F486E080938E011092DD018AE049
:1037700080938F019093DE018AEA8093F10380E0C9
:1037800008958091DE01813071F480918F01815024
:1037900080938F018F5F39F48091F1038FB910927C
:1037A000DE0181E0089581E00895CF93DF93C0E0CA
:1037B000D0E0E0919001F0919101EC0FFD1F80812C
:1037C0000E94F9112196C730D10599F78DE00E942A
:1037D0001D12DF91CF910895FC0188279927E89465
:1037E00021912032E9F3293010F02E30C8F32B322A
:1037F00041F02D3239F4689404C00E94321C820FCB
:10380000911D219120532A30C0F31EF4909581958B
:103810009F4F0895FB01DC0101900D920020E1F71C
:103820000895FB019F01E8944230C4F04532B4F49E
:103830004A3029F497FB1EF4909581959F4F642F91
:1038400077270E94631C805D8A330CF0895D819329
:10385000CB010097A1F716F45DE251931082C901E4
:103860000C943A1C7AE0979F902D879F802D910DA4
:1038700011240895DC01FC01672F71917723E1F792
:10388000329704C07C916D9370836291AE17BF072D
:10389000C8F30895991B79E004C0991F961708F0A2
:1038A000961B881F7A95C9F78095089587FB082E87
:1038B000062687FD819567FD6195ECDF0EF49195F5
:1038C00007FC81950895AA1BBB1B51E107C0AA1FE5
:1038D000BB1FA617B70710F0A61BB70B881F991FB1
:1038E0005A95A9F780959095BC01CD01089597FB55
:1038F000092E07260AD077FD04D0E5DF06D0002088
:103900001AF4709561957F4F0895F6F7909581951B
:083910009F4F0895F894FFCFCA
:103918000101030E0786010E0C5C00000A0000443A
:10392800000023002300546466536365526200510B
:1039380061005060005060005161005262005363A2
:10394800655464666768696A6B6B6A6968670000D2
:103958000053536353534103F701BF030D0A20205B
:10396800005048004348000A1D000000000000689D
:10397800656C70200D0073686F772049440D0073E3
:10398800686F772076657273696F6E0D0049442001
:103998003D2000302E392E372E302E310D000907EC
:0239A800910389
:00000001FF
